:100000004828000000000000A8000308A9004030B4
:100010008606A003031D1428A1030F3021052730F5
:1000200003192830A00026140B1129088300280882
:1000300009000000000000000000000000000000B7
:1000400000000000000000000000000000000000B0
:1000500000000000000000000000000000000000A0
:100060000000000000000000000000000000000090
:100070000000000000000000000000000000000080
:100080000000000000000000000000000000000070
:100090000630A2000930A300A401831603138030A8
:1000A00081003830850000308600831207309F00C1
:1000B000A0308B0007308500FF3086003230A5006D
:1000C0002830A0000430AB00A601A701AE018101D9
:1000D000B0018321261C7228E020FB20271E7228F5
:1000E0002712AF21B001A71A9228FF302406261D3F
:1000F0007B28FE30A7208600FE30AE20B720FF30E0
:10010000A71D2306A619A7208600FD30AE20B72024
:10011000FF30A71D2206261AA7208600FB30AE203E
:10012000B7206A28FF302C068600FE30AE20B720AC
:10013000FF302C1BFE308600FD30AE20B720FF3094
:10014000A718EF308600FB30AE20B7206A28AA003F
:1001500019302502FF3003182A080800AF00850572
:10016000C1202F09051EB528B000850408002B18F2
:10017000C028AB183F302B19FF30AA00AA0BBE28AD
:1001800008001830AA00AA0BC32808002408031D81
:10019000DF282D080319D62803302305031DDF2887
:1001A000AD03A71CD528A50AD628A503073022052C
:1001B000031DDF282308031DDF282C08AD000800DD
:1001C0002610A50BFA283230A500C6203C30A40A20
:1001D0002406031DFA28A40027163C30A30A230690
:1001E000031DFA28A300A6141830A20A2206031D34
:1001F000FA28A200080001302505031D7729301DCB
:100200001929A7197729A61A7829A616A71E0D2934
:10021000A71291210F30A6057729AE01A61D13293B
:10022000A61126167729261E172926127729A61524
:100230007729A612B01C4429A7197729261B7729EC
:100240002617A61D2929A30A3C3023060319A3005B
:100250007729261E3129A20A183022060319A20086
:100260007729A71E3E29A7183A2978302C06031DA6
:10027000AC0A7729AC030319A7107729AB0C031C30
:1002800077290430AB0077292613301C7629A61B6A
:100290007729A617A61D5329003023063B30031DDE
:1002A0002303A3007729261E5C290030220617307D
:1002B000031D2203A2007729A71E6929A71C65290F
:1002C00078302C06031DAC0A7729AC030319A71458
:1002D000772926196D2926157729A71D7229A711B7
:1002E00026117729A7150430AB007729A61308003B
:1002F000A6197729261A7729A71A7729AE0A2E1F59
:100300007729A7167729831600309B001C141A083A
:100310008312AC00AC1F8E29A714AC132C08AD00BF
:1003200008002C08AD00A718803E83169A00003004
:100330009B001C158B138B1B9B2955309D00AA30ED
:100340009D009C149C18A2298B171C118312080075
:1003500000000000000000000000000008000A305B
:100360009F00831684309F008312A8211F1BBC2985
:10037000A71526150430AB0000309F0007309F0002
:02038000080073
:02400E00291F68
:104200000100FF00FF00FF00FF00FF00FF00FF00B4
:10421000FF00FF00FF00FF00FF00FF00FF00FF00A6
:10422000FF00FF00FF00FF00FF00FF00FF00FF0096
:10423000FF00FF00FF00FF00FF00FF00FF00FF0086
:10424000FF00FF00FF00FF00FF00FF00FF00FF0076
:10425000FF00FF00FF00FF00FF00FF00FF00FF0066
:10426000FF00FF00FF00FF00FF00FF00FF00FF0056
:10427000FF00FF00FF00FF00FF00FF00FF00FF0046
:10428000FF00FF00FF00FF00FF00FF00FF00FF0036
:10429000FF00FF00FF00FF00FF00FF00FF00FF0026
:1042A000FF00FF00FF00FF00FF00FF00FF00FF0016
:1042B000FF00FF00FF00FF00FF00FF00FF00FF0006
:1042C000FF00FF00FF00FF00FF00FF00FF00FF00F6
:1042D000FF00FF00FF00FF00FF00FF00FF00FF00E6
:1042E000FF00FF00FF00FF00FF00FF00FF00FF00D6
:1042F000FF00FF00FF00FF00FF00FF00FF00FF00C6
:00000001FF
